:030000000219FDE5
:03000B000200A848
:03002B000201616E
:03005B000202F2AC
:030073000202DFA7
:1000800002030406080C10182030406080040608A3
:100090000C10182030406080A0C00003070F1F051F
:1000A000050D050305030302C2AFC0D0C0E0206206
:1000B00014E5256009E473E525F4F58AD262D0E001
:1000C000D0D0D2AF3285268AC262E526F4603630BF
:1000D000682C20720DD0E0D0D0C282C286C287D2F6
:1000E000AF32C282C286C287206F13206510740AA5
:1000F000D5E0FDE57BB40104429001FE4280D0E0F2
:10010000D0D0D2AF32758A00C28DD26201FE01B763
:10011000306805206502D28201B73068052065028B
:10012000D28601B7306805206502D28701B7C28147
:1001300030680A2065077406D5E0FDD28201B7C297
:100140008330680A2065077406D5E0FDD28601B7C2
:10015000C29030680A2065077406D5E0FDD2870199
:10016000B7C2AFC2AD53E6EFC0D0C0E0D2D3D2AF7A
:10017000C2CEE52A600720744F152A21C87800797D
:100180000020742EE580307E01F430E50278FF53C4
:10019000DACF207E0343DA20307E0343DA10C2D860
:1001A000C271E580307E01F430E50279FFC3E89941
:1001B00070CB306103752A18207403752A18885C87
:1001C000D270E86003755F0020740DE52B600415A4
:1001D0002B21D843DA01C2D8207002414BA85C2001
:1001E0006102C270207431C3E894F0400374F0F8E7
:1001F000E8C4540F28F87984B703024118C313C325
:10020000138721200802C313200A06C3C898F841A7
:100210001828F8500374FFF8C3E895655003E565A6
:10022000F88822E52D54066022206B1FE536C33383
:10023000C333F8E564C313C313F9C395224002899D
:1002400022E82522F52250037522FF852224A824C6
:10025000C3E52495614002A8618825E566700241E6
:100260008FC3E8AA669A5003E8FAE4F9EAC333FBBD
:10027000E568F45B29400D2567F8E56760021567BE
:10028000400B418F0AC3E5679A5002056778FF88E3
:1002900026C26FC3E52694F84002D26F20CF0AD061
:1002A000E0D0D043E610D2AD32C2CF053A7801E5B6
:1002B0002A6005307402152AC3E55C940140057577
:1002C0005F0041D5756000756900E55F2401F55F49
:1002D0005003755FFFD0E0D0D043E610D2AD32C2FC
:1002E000AF53E67F7592FA7593FFC260759104D2A1
:1002F000AF32C2AF53E6EFC2ADC0D0C0E0C0F0D263
:10030000D3D2AFA8FBA9FCC2D8307102615953DA2D
:10031000CF207E0343DA10307E0343DA20D271E52A
:1003200080307E01F420E502613088278928A1868B
:1003300053DACF207E0343DA20307E0343DA10C243
:10034000D8C271307402A1727800E580307E01F469
:1003500030E502A172885CA15A53DACF207E0343B4
:10036000DA20307E0343DA10C271206102813253F9
:10037000DACF207E0343DA10307E0343DA20C2D87E
:10038000D27188578958C3E89555F8E99556F97B95
:10039000007E087A00C3E8948CE994005005755BF0
:1003A000008124882178A2E6A8216055C3E894C87A
:1003B000E994005008E4D2E4FB7A0A61FFC3E894B0
:1003C00068E994015008E4D2E3FB7A0F61FFC3E8C7
:1003D00094D0E994025008E4D2E2FB7A1E61FFC394
:1003E000E894A0E994055008E4D2E1FB7A3C61FF6F
:1003F000C3E89498E994085008E4D2E0FB7A787E48
:1004000000C3E89559FCE9955AFD30E70AECF4245D
:1004100001FCEDF43400FD755B00C3EC9AED9E50D9
:1004200003755B018859895A855755855856780256
:10043000A15AC3E89527F8E99528F9307C02A13E36
:10044000307B02A13E307A02A1372075028155E946
:10045000FDE8FC8174E9C313F9E813F8307902A1CF
:1004600037E9C313F9E813F8307802A137E9C31369
:0E047000FDE813FC20612CC3EC941CED9402FB
:10047E004002818BED701EC3EC94C850180529E51F
:10048E002970021529C3E529940A5002A172755CE0
:10049E0000D270A172E529600215297888E6F974F8
:1004AE0000207F087896B90302789EE624FAFEE4CF
:1004BE003400FFC3EC9EFCED9FFD9208B90310A221
:1004CE00085007207609D27681DD307602C276A2F8
:1004DE00085016B9030DECF42401FCEDF43400FDC4
:1004EE000204F778007900A13EB90315EC33FCED58
:1004FE0033FDC3EC940AFCED9400FD50047C007DAA
:10050E0000C3EC94FFED9400400678FF7900A13E05
:10051E00EC8572F0A4C5F0A2F733F879004003021F
:10052E00055A78FF790002055AE9C313F9E813F862
:10053E00307C0EE9600278FFC3E81338F8E434002B
:10054E00F9C3E894FFE99400400278FF885CD2700A
:10055E00206102A172741FF4552F4BF52FC274EB5C
:10056E007002D274752A18307403752A0A3061022B
:10057E00A18620740353DAFE207403752B06D0F087
:10058E00D0E0D0D0D2AD43E6103279010205B67973
:10059E00030205B6790A0205B6791E0205B679641C
:1005AE000205B679C80205B67817E4D5E0FDD8FA8B
:1005BE00D9F6227A147B780205DD7A107B8C02053F
:1005CE00DD7A0D7BB40205DD7A0B7BC80205DDE515
:1005DE0073D5E001227902E4C283D5E0FDD286D53F
:1005EE00E0FDC286D5E0FDD283D5E0FDE920E00234
:1005FE00D28230E002D287E573D5E0FDE920E00239
:10060E00C28230E002C2877496D5E0FDD9C9EAF8FD
:10061E00D5E0FDD8FBDBB8C28322C37C007D00751C
:10062E00F00005F0EA33FAEB33FB50F6EB13FBEA7E
:10063E0013FAC3E9FFE8FEE89AF8E99BF95004EFD4
:10064E00F9EEF8B3EC33FCED33FDD5F0DFEDF9EC5C
:10065E00F822E889F08A20D2D4F8A9F07B0030F78E
:10066E000B7BFFF42401F8E9F43400F9E88520F05F
:10067E00A4ADF0F8E98520F0A4AFF0FEED2EF974EC
:10068E00003FFA7C04C3EA13FAE913F9E813F8DC25
:10069E00F48BF030F70AE8F42401F8E9F43400F9A9
:1006AE00E889F0C2D4F8A9F02222C3E54113F9E596
:1006BE004013F8C3E54498F8E54599F9500CC3E8A2
:1006CE009480E994FF40160206EFC3E8947FE99404
:1006DE000050030206EF787F79000206EF788079EA
:1006EE00FF8849894A22E5492546F8E54A3547F902
:1006FE00854A20E4300701F43548FA30E709C3EAA9
:10070E0094F0401502072DC3EA940F500302072DF3
:10071E0078FF79FF7A0F02072D780079007AF0C3FF
:10072E00E5249561500AC374019524500B02074BC2
:10073E00E54A20E70E02074BE54A30E70688468970
:10074E00478A482278A5E6FAC3E54933F8E54A33E5
:10075E00F9D160E930E70BC3E89480E994FF4013C8
:10076E00E185C3E8947FE994005002E185787F79B2
:10077E0000E185788079FFE820E715C3E52398F836
:10078E004009C3E8940140030207AC78010207ACAC
:10079E00E8F424012523F840030207AC78FF884BC8
:1007AE002278A6E6FAA847A948D160E930E70CC33B
:1007BE00E89401E994FF40160207E0C3E894FFE9CC
:1007CE00940050030207E078FF79000207E07801F9
:1007DE0079FFE920E715C3E54B98F84009C3E89483
:1007EE000140030208077801020807E8F4240125F6
:1007FE004BF8400302080778FF88242278FF20690F
:10080E002879A1E76023E541601F74FF8541F084DC
:10081E008539F0306A0375F005A4F8C5F0600278EA
:10082E00FFC3E895645002A864886322C3E5409430
:10083E0040E5419401E563500314014B046002F559
:10084E0063220208532275E890227883E6FF30ED8A
:10085E00F9A8BDA9BE0570C3E57094084052757025
:0F086E0000E9FA79A0E76044EA7007E571601BC2
:10087D0002088CC3E895716010E5715006600C1488
:10088D000208980460F9020898E571F571C3946740
:10089D00401B7561C0C394044013756180C39404FB
:1008AD00400B756140C39404400375610075BB0B2B
:1008BD0022E561F460020561E570B4070375BB10B4
:1008CD0022743279A787F0A4C5F0A2F733F8C3E8F4
:1008DD0095614002A861882288248825882688642D
:1008ED00227540007541F022C2AF75C820A8CCA971
:1008FD00CDAA3A30CF010A75C824D2AFAB3BAC3C80
:10090D00883B893CC3E89BF8E99C206908F930666F
:10091D000241062160AD3D8A3DF9EA9DFA600678F7
:10092D00FF79FF2145AE3EAF3F8B3E8C3FA83BA9E3
:10093D003CC3E89EF8E99FF9C3E54113FBE540137D
:10094D00FAE82AF540E93BF54150067540FF75413F
:10095D00FF21ADAA40AB41AC40AD417E047F02C347
:10096D00EB9404400D1E1FC3EB94084005206A0252
:10097D001E1FC3ED13FDEC13FCDEF7C3EA9CFAEB6F
:10098D009DFBEF6009C3E913F9E813F8DFF7EA28D7
:10099D00FAEB39FB8A408B4150067BFF8B408B4134
:1009AD00C3EB94025002D2663069047F0321D878DC
:1009BD0092E6FFC3E537948240110FC3E53794A04B
:1009CD0040010FC3EF940640027F057E02E541C44E
:1009DD00540FF9E541C454F0F8E540C4540F28F81C
:1009ED00C3E89EFAE99400FB4009C3EA9402EB9434
:1009FD000050047A02E4FB4152AA40AB41EBC4FE25
:100A0D00EAC4540F4EFCC3EA9CFAEB9400FBC3E816
:100A1D0013C313F8EA28FAEB3400FB8A408B41C369
:100A2D00EB94024002C2667802EBC4FE7B00EAC47E
:100A3D00540F4EFAC3EA98FA4005C3940250027A55
:100A4D00027892E6FF3060024152855192855293B1
:100A5D00D26043E680C3E49AF8E49BF93066024124
:100A6D00DEE8FAE9FBD3E913FDE813FC885189525E
:100A7D00C3EF94036038EF20E00DE82CF8E93DF961
:100A8D00ECFAEDFB020AA7E828F8E939F9C3E824E6
:100A9D0002F8E93400F97AFE7BFFC3EF9403400EB0
:100AAD008A538B54884D894E8C4F8D5061128853CB
:100ABD0089548A4D8B4E8C4F8D503069127553F081
:100ACD007554FF754FF07550FF7551F07552FF61FC
:100ADD0012E8FAD3E813FC8851C3EF94036020EFBA
:100AED0020E007E82CF8ECFA41FEE8282402F87A19
:100AFD00FEC3EF940340088A53884D8C4F611288D2
:100B0D00538A4D8C4FE568C3335002646BF56830E2
:100B1D006002611C753402D26043E680E52D5406F7
:100B2D006034A840A941C3E913F9E813F8C3E913E8
:100B3D00F9E813F8306904E92440F9C2AF53E67FB0
:100B4D00759100C3E498F594E499F595759104D2E7
:100B5D006043E680D2AF22D2647543007520003029
:100B6D006C03752040020B83D264754300752040E1
:100B7D00306C0375200078017901206620E52D5435
:100B8D00066002C2647914E541C313700104F8C311
:100B9D00941440027814306904781B791B2060107E
:100BAD00E543600C306903D53404D26D812D712479
:100BBD000543E5BF5440B52002811730690908C3CC
:100BCD00E89940011861AA20640A08C3E899400217
:100BDD00618361AAC264C2AF53E67F75910030662E
:100BED00127594007595F8759104D26043E680D224
:100BFD00AF6183E5417EFFC3334005C3334001FE42
:100C0D00C3E49E759400F59561F4C3E533940150EA
:100C1D000261833064026183D802812B61AAC26DA7
:100C2D00C2AF53E67F7591008553948554957591A8
:100C3D0004854D92854E93D26043E680D2AFE52D6B
:100C4D0054066008206A020533020C69306D0D20D0
:100C5D006C0A206407158115810215412278003038
:0E0C6D0064027801E53775F007A4F9E5F02878
:100C7B00F5F0E9A2F013A2F113A2F213F537C39426
:100C8B00785003753778C3E53795384008D265C27D
:100C9B0082C286C28730600281A0854F92855093B5
:100CAB00D26043E68022207D16C2AF754202C2831A
:100CBB00D281306202D287D2AF75AA23020EA1C2B3
:100CCB00AF754202C283D290306202D282D2AF752C
:100CDB00AA23020EA1307243207D20C2AF754203BE
:100CEB0090013F757B08C287C290306204D2868127
:100CFB00FED283D2AF75AA24020EA1C2AF754203F6
:100D0B0090013F757B08C282C281306204D286A1FA
:100D1B001ED283D2AF75AA21020EA1207D17C2AFBE
:100D2B0075420390011AC287306202D286D2AF7528
:100D3B00AA24020EA1C2AF75420390011AC28230DF
:100D4B006202D286D2AF75AA21020EA1207D16C2F5
:100D5B00AF754204C281D290306202D286D2AF7597
:100D6B00AA21020EA1C2AF754204C290D281306299
:100D7B0002D286D2AF75AA24020EA1307243207D17
:100D8B0020C2AF75420590012E757B02C286C283CD
:100D9B00306204D282A1A4D281D2AF75AA23020EF3
:100DAB00A1C2AF754205900150757B01C286C2830B
:100DBB00306204D287A1C4D290D2AF75AA23020E9F
:100DCB00A1207D17C2AF754205900110C28630621B
:100DDB0002D282D2AF75AA23020EA1C2AF75420511
:100DEB00900124C2863062EBD287D2AF75AA230260
:100DFB000EA1207D16C2AF754206C290D28330621F
:100E0B0002D282D2AF75AA24020EA1C2AF754206DE
:100E1B00C281D283306202D287D2AF75AA21020E71
:100E2B00A1307244207D20C2AF75420190015075F4
:100E3B007B01C282C281306204D287C14AD290D276
:100E4B00AF75AA21020EA1C2AF75420190012E759A
:100E5B007B02C287C290306205D282020E6BD281B6
:100E6B00D2AF75AA24020EA1207D17C2AF75420125
:100E7B00900124C282306202D287D2AF75AA2102BE
:100E8B000EA1C2AF754201900110C287306202D22F
:100E9B0082D2AF75AA24C2652290010E757B00C267
:100EAB0082C286C287C281C283C290C2622278800C
:100EBB0076FF0876FF0876FF0876FF08760308763C
:100ECB000408760A087603087601087601788C7692
:100EDB00010876FF0876FF0876FF0876FF0876FF95
:100EEB000876030876FF0876FF0876FF0876250854
:100EFB0076D00876FA0876FA0876040876FF087634
:100F0B000108760008767A0876FF087601087601E4
:100F1B00087600087603087600227887E6FFC2720F
:100F2B00BF0302D2727888E6C394036008C27DE6E1
:100F3B0030E102D27DC27E7889E630E102D27EC3F7
:100F4B00EF94026008758E01D273020F5D758E00EF
:100F5B00C273227880E6149000809378A5F678818E
:100F6B00E6149000809378A6F67886E61490008DB0
:100F7B009378A7F67886E6F539C394025003753952
:100F8B0002789CE67538FFB402037538A0B40303EE
:100F9B0075388278A3E61490009A93F566D1A42253
:100FAB00227896E6FA7897E6FB7888E6B40305C3D1
:100FBB00EB940EFB307F047A007BFFC3EB9AFCC3F0
:100FCB00948250027C827572000572EC8572F0A4DB
:100FDB00C3E5F0947D40F222D27FF1AC1205A7124B
:100FEB0005A77A007B007C1012059DE55C2AFA743C
:100FFB00003BFBDCF37C04C3EB13FBEA13FADCF7DB
:10100B00FEC27F120FAC22757C00757D00E5EF20D0
:10101B00E6037520000520903FFFE5201460069045
:10102B001FFF1460009304600375EF167597DE7550
:10103B0097AD7581C043FF8012059875EF0675A9B2
:10104B0000E5C7240220E70DF521E5B120E0068578
:10105B0021C743B101120EA475803175A4CE75F171
:0D106B00FF75D4DF7590FE75A50175F2E1EB
:1010780075D50075A60175E34075E201120EA4E46A
:10108800F8F6D8FD756801120EB91215927898868F
:1010980073753001C2AF1205B11205C11205A7124E
:1010A80005C81205A71205CF1205A71216BB12050F
:1010B800B11205B11205ACC2AF757C00757D007820
:1010C800FA79FA308507D9FBD8F7021C00120F25E8
:1010D800120F5E120FAB120FAC78988673120EA423
:1010E80075881075890275C82475910475D840757E
:1010F800A82275B80275E690759B80759D0075BF2E
:101108008075AB0075D10C75BC5975BB0B75E88043
:1011180075B201120598D2AF12085075360053DA2D
:10112800CF207E0343DA20307E0343DA1043DA010E
:10113800C2D8C2711205B1D2617B037A0CE55B702B
:10114800077A0CDB030210BF1205A72070030210F8
:10115800BFC270E55CC3940240E1E52F541F855E71
:101168005DF55EB55DD5DAD5C26153DACF207E0371
:1011780043DA20307E0343DA10C2D8C27178A2E67F
:101188007008D274E52F54E0F52FC2757529001246
:1011980005AC307409C3E529940A4002D2751205DA
:1011A8009D78023074027800C3E55C9840F0C2AFC5
:1011B8001205C11205C11205C1D2AF1205B1754C95
:1011C800007888E6B4030241C512059D788CE6C311
:1011D800940150030212C5E530C394015003021272
:1011E800C5757CA5757DF1207435C3E55C94FF5009
:1011F800030212C5C2AF1205D6D2AF1205ACC3E5C1
:101208005C940150EFC2AF1205C11205A21205C1CC
:10121800D2AF1205ACC3E55C94FF40E90217407FEA
:1012280005D27F120FAC1205ACC2AFC27F120FAC51
:10123800AE5CC3E55C947FD2AF500241D5120598ED
:10124800C2AF1205D6D2AFDFD8120FE3C3EE9405B2
:101258007897F61205B11216C37F0AD27F120FAC27
:101268001205ACC2AFC27F120FACAE5CC3E55C9492
:101278007FD2AF50E4120598C2AF1205C11205A281
:101288001205C1D2AFDFD4120FE3EE24037896F62D
:10129800F87997E7C394824003985006E824827847
:1012A80097F61205B11215E01216F21205AC120FDC
:1012B800ACC3E55C94FF500221E9021740757C003D
:1012C800757D00C3E55C954C4003855C4C1205AC0C
:1012D80078017988E7B403027805C3E55C98400291
:1012E80021C9C2AF1205D61205D61205D6D2AF1241
:1012F80005B1753000E4F531F5320531E531F470AA
:101308003F0532789AE67819146012783214600D25
:10131800787D14600878FA146003753200C3E532EA
:1013280098401D120EA4120598153275310078994F
:101338008673C2AF1205D6D2AF789886731205AC01
:101348001205A2E52A700530740201BF78012074E5
:10135800027806C3E55C9840A17888E6C3940360E8
:10136800031205ACE52A70030210BFC2AF120EA427
:10137800E4F522F523F524F525F526F567D2AF78AF
:1013880085E6C333F565E4F544F545F546F547F5D7
:1013980048F570F52CF52DF53775700875BB1012EA
:1013A800059812085430EDFDA8BDA9BEE97001F8F2
:1013B800887112085875700875BB10120F25C2AFD6
:1013C8007561FF1208CE852261852262852263D26B
:1013D800AF7522017524017525017526018560699F
:1013E800756A017888E6B40307C27D307602D27D3B
:1013F800D268D269753300120DFD120E2C1208EE58
:101408001208F51208EE1208F51208EE120B751202
:1014180006B7120C6A120CB11208F5120B64306E82
:10142800031206B820660312080A30660312083A47
:10143800120C6A120CE01208F5120B75306E0312CA
:1014480006F4120C6A120D571208F5120B64306E6E
:1014580003120752120C6A120D861208F5120B7548
:0F146800306E031207AF120C6A120DFD1208F559
:10147700120854120B64120C6A120E2C120858121E
:1014870008F530692F856461856462856069756ACE
:101497000179187A0CC3E53399400CC269D26A8A7C
:1014A700357561FF0214BBC3E55C94014003021468
:1014B70014021549306A25206C22E535147006C2DE
:1014C7006AD26B8114F535C3E55C940140030214BD
:1014D700147888E6C39403600302154975360078CB
:1014E7008279A4E760027803C3E55F9850543074AB
:1014F70004E52A604D7888E6B40317207D05207639
:1015070007A119307602A119206C07D26C85646196
:10151700815378F0306C058564617820C3E5419884
:1015270050028114306C1BC26CC27D307602D27DB2
:10153700D26A75351285646181140536E55C6002EF
:10154700A14C753600C2AF120EA47887E6FE76026C
:10155700120F257887EEF6E4F522F523F524F52515
:10156700F526F565752C00752D00D2AF1205AC1266
:101577000EA478A4E66006D282D286D28730740998
:10158700C3E5369404400201BF41FD901A0D78204F
:10159700121622E520B45A0CA3121622E520B4A590
:1015A700030215C0757CA5757DF1120EB91215E001
:1015B700757C00757D000215DF901A0378807B0A21
:1015C700121622A308DBF9901A0F788C7B191216D2
:1015D70022A308DBF9901A2822C2AF121665121649
:1015E70042901A00740E121627A37409121627A325
:1015F7007415121627901A0378807B0A121626A3F1
:1016070008DBF9901A0F788C7B19121626A308DBD2
:10161700F9121678121656901A2822E493F622E643
:10162700438F01538FFDFFC3E583941C400122EFD5
:10163700857CB7857DB7F0538FFE22438F02438F9A
:1016470001857CB7857DB7901A0DF0538FFC2290EA
:101657001A0D745AD127901A0E74A5D127227A3001
:1016670079D07820901A40D122E520F709A3DAF73C
:10167700227A3079D0901A40E7D12709A3DAF922E4
:10168700AB74A875BB01027984BB02027985BB03E1
:10169700027986BB04027992BB05027987BB0602F1
:1016A70079A3BB0702799CBB08027988BB09027939
:1016B70089E8F7227C051205B1DCFB22C2AF1205CF
:1016C700C11205C81205CF1205D61205A21205C10F
:1016D7001205C81205CF1205D61205A21205C112AE
:1016E70005C81205CF1205D6D2AF22C2AF1205D652
:1016F7001205CF1205C81205C11205A21205D6128E
:1017070005CF1205C81205C11205A21205D612058A
:10171700CF1205C81205C1D2AF22AE74AF75C2AFE2
:101727001205C11205C11205C11205A2DEF212058A
:10173700D61205A2DFF8D2AF22D1C3D1BBD1BB7578
:101747007401757501757600F1217C05AD5C120594
:10175700B1C3ED955C70F5C3E55C9401400AC3E540
:101767005C94FF403202177CD187B1E0D1C3C2AF8E
:1017770075EF16D1BBDCD50576C3E5769403500229
:1017870080C6D1BB0575E5741490009F93F808C314
:10179700E57598500280AED1BBD1BB0574C3E57423
:1017A700940A5002809C120EB9B1E0C2AF75EF16D1
:0217B700D1BBA4
:0319FD00021012C3
:101A00000E0915FFFFFFFF03040A0301015AA50198
:101A1000FFFFFFFFFF03FFFFFF25D0FAFA04FF01DE
:091A2000007AFF0101000300FF40
:101A4000234D5232355F3135412320202020202084
:101A500023424C48454C492346383530232020202A
:101A60002020202020202020202020202020202076
:101C0000C2AFC2D37597DE7597AD7581C075A90057
:101C100043FF80752438752503B1DB7529A5752A26
:101C2000F175E34043F12053A4DF75D4FFD2857DE5
:101C3000FA780379E67C10752200752300901DE880
:101C40007B0675249875250130850281482085081A
:101C5000D8FBD9F9DCF781BA308508D8FBD9F9DC93
:101C6000F781BAB19BE493A3C39A6004DDC381BA40
:101C7000DBDBB18D600281317B08E493FAA3B16EA6
:101C8000DBF87A30B16E752200752300B18DEAFC65
:101C9000EBFDC3ED94FE400EB18D8A278B28ED300D
:101CA000E0048A828B83B18D7AC270D8C3ED94FE32
:101CB000601950CEBD0029EC600F7520007521FF22
:101CC000752900752A000200008100A827A92808AC
:101CD00009D804D90281DDB191EAF281D10D81A642
:101CE000C3ED94035051EDA2E092007AC5C3E582A2
:101CF0009400E583941C508C200010438F02438F86
:101D0000018529B7852AB7F0300027A827A9280818
:101D100009438F01538FFDD804D902A132C3E58353
:101D2000941C4003A3A117E28529B7852AB7F0A325
:101D3000A117538FFC81827AC1BD030CE493A3FAEF
:101D4000B152DCF8B14A81828184AA22AB23B16E00
:101D5000EBFAEA6222752608C3E52313F523E52290
:101D600013F52250066323A0632201D526EAB1DBD6
:101D7000B1DB75260AEAF4200102D285300102C2E5
:101D800085B1DBC3134002C201D526EB22B191EA33
:101D9000FB208502A191308502A196752608AE240C
:101DA000AF25C3EF13FFEE13FEB1DFB1DBC3EA13C0
:101DB0003085024480FA30E703632201C3E5231330
:101DC000F523E52213F52250066323A0632201D5F3
:101DD00026D9E52265236523F52222AE24AF250E00
:101DE0000FDEFEDFFCD20122424C48656C693437BD
:061DF0003164F850060109
:00000001FF
